:100000002CC050C049C248C24DC04CC04BC04AC0B1
:1000100049C048C047C0F6C145C044C043C042C003
:1000200041C000003900360000003A0037000000EF
:100030003B0038000101010101010101020202013E
:1000400002040810204080040201000000000004A7
:100050000302010000009803010411241FBECFE534
:10006000D1E0DEBFCDBF10E0A0E6B0E0ECEAF8E002
:1000700002C005900D92A83CB107D9F721E0A8EC89
:10008000B0E001C01D92A433B207E1F710E0CCE26A
:10009000D0E003C02197FE01F7D3CB32D107D1F7CF
:1000A00073D2F8C3ADCF0895AF92BF92CF92DF92D3
:1000B000EF92FF920F931F93CF93DF936C017B011D
:1000C0008B01040F151FEB015E01AE18BF08C017AE
:1000D000D10759F06991D601ED91FC910190F08121
:1000E000E02DC6010995892B79F7C501DF91CF91E4
:1000F0001F910F91FF90EF90DF90CF90BF90AF9046
:10010000089590E0FC01E65BFF4F3491FC01E15C57
:10011000FF4F2491FC01EC5CFF4FE491EE23B9F01A
:10012000332329F0323019F198F43130E1F0F0E066
:10013000EE0FFF1FE25DFF4FA591B4918FB7F894CA
:10014000EC91611117C020952E232C938FBF089539
:10015000333029F0343059F78FB58F7D02C08FB519
:100160008F778FBDE4CF80B78F7780BFE0CF80B728
:100170008F7DFBCF2E2BE9CFCF93DF9390E0FC0157
:10018000E15CFF4F24918C5C9F4FFC01849188239C
:10019000D1F090E0880F991FFC01E85DFF4FA59119
:1001A000B491FC01E25DFF4FC591D49161110EC085
:1001B0009FB7F8948C91E22FE0958E238C93288141
:1001C000E223E8839FBFDF91CF9108958FB7F89422
:1001D000EC91E22BEC938FBFF6CF3FB7F894809170
:1001E0000D0190910E01A0910F01B091100122B765
:1001F00008B600FE05C02F3F19F00196A11DB11DE4
:100200003FBFBA2FA92F982F8827BC01CD01620FBD
:10021000711D811D911D43E0660F771F881F991F77
:100220004A95D1F708958F929F92AF92BF92CF9245
:10023000DF92EF92FF92D1DF4B015C0180EDC82E7F
:1002400087E0D82EE12CF12CC8DF681979098A09DA
:100250009B09683E734081059105B0F321E0C21A05
:10026000D108E108F10888EE880E83E0981EA11CF1
:10027000B11CC114D104E104F10431F7FF90EF90F7
:10028000DF90CF90BF90AF909F908F900895209176
:100290001301309114012817390771F4909111015D
:1002A00080911201981741F0E0911101F0E0E853BC
:1002B000FF4F808190E008958FEF9FEF0895EF92B8
:1002C000FF920F931F93CF93DF93DC015C96ED9029
:1002D000FC905D97E114F10479F481E090E01396CD
:1002E0009C938E93129790E080E0DF91CF911F91C5
:1002F0000F91FF90EF9008955196ED91FC915297D8
:1003000050968C915097982F90950FB75E962C91A0
:100310005E97122F127021FD6095F89420811123B1
:1003200019F1282B2083E7012197F1F728E0462FC8
:1003300050E0308160FF1AC0382B3083E7012197ED
:10034000F1F7BA0175956795215089F7112381F06E
:100350008081892380830FBF5C968D919C9101974A
:10036000F1F781E090E0C1CF2923DCCF3923E5CF3D
:100370009081892BEFCF2091130130911401281720
:10038000390769F4809112012091110190E0805C9D
:100390009F4F821B910960E470E04FD2089590E076
:1003A00080E0089520911301309114012817390736
:1003B000B9F49091110180911201981789F0E091A0
:1003C0001101F0E0E853FF4F80812091110130E0EE
:1003D0002F5F3F4F2F7333272093110190E0089533
:1003E0008FEF9FEF089590E080E00895FC01019069
:1003F0000020E9F73197AF01481B590BBC0185E19B
:1004000091E052CE1F920F920FB60F9211242F93AC
:100410003F938F939F93AF93BF93809109019091E6
:100420000A01A0910B01B0910C013091080126E066
:10043000230F2D3758F50296A11DB11D20930801F9
:100440008093090190930A01A0930B01B0930C01D2
:1004500080910D0190910E01A0910F01B0911001BA
:100460000196A11DB11D80930D0190930E01A093E3
:100470000F01B0931001BF91AF919F918F913F9168
:100480002F910F900FBE0F901F90189529E8230F02
:100490000396A11DB11DD2CF1F920F920FB60F92DE
:1004A00011242F933F934F935F936F937F938F9379
:1004B0009F93AF93BF93EF93FF93E0911301F0915C
:1004C0001401309749F0A685B7858585968D91FFF3
:1004D00014C09C918923A1F4FF91EF91BF91AF913A
:1004E0009F918F917F916F915F914F913F912F914C
:1004F0000F900FBE0F901F9018959C91892361F764
:10050000A389B4899C918589809589238C93868958
:1005100097890197F1F7608D718DA685B78555850F
:1005200038E020E0CB010197F1F7822F90E095951C
:100530008795282F4C91452309F02068315091F779
:10054000868D81FD20958091120190E001968F7338
:10055000992730911101381799F0A0911201B0E05C
:10056000A853BF4F2C9380931201828D938D0197D6
:10057000F1F7A389B4898C919589892B8C93ACCFA1
:10058000868D8160868FF1CF789480B7826080BF3E
:1005900080B7816080BF83B7826083BF83B781608B
:1005A00083BF89B7816089BF1EBC8EB582608EBD56
:1005B0008EB581608EBD8FB581608FBD329A319AC4
:1005C0003098379A60E081E0D7DD61E080E0D4DDEB
:1005D0001092300110922F0110922E0110922D01D5
:1005E00010922C0110922B018DEC90E0909332012F
:1005F00080933101909121019B30C8F525E530E0D1
:1006000030932C0120932B012BEC30E030932E0102
:1006100020932D0120E930E03093300120932F0109
:100620008BB720E1983008F020E2822B8BBF22E3C9
:1006300030E0983030F020E430E09B3010F030E0D3
:1006400020E03093290120932801492F50E0983071
:1006500008F064C081E001C0880F9A95EAF78093A2
:100660002A0180913101909132010197F1F7809137
:100670002F0190913001892B49F1E0911301F09104
:10068000140181E0E531F80709F1309739F0A389C9
:10069000B4899C918589809589238C9380913301BD
:1006A0008E7F80933301109212011092110185E127
:1006B00091E09093140180931301E0912801F0914F
:1006C0002901808190912A01892B808382E790E023
:1006D0008DDE80E890E08ADE85E990E087DE83EABF
:1006E00090E084DEA0DD81EB90E080DE9CDD61E0C7
:1006F00088E042DD61E088E004DDD0E0C0E085E133
:1007000091E039DE892BD9F385E191E04BDE21962A
:1007100061E0C0FD60E088E0F4DCF1CF2AE030E089
:10072000241B350B81E001C0880F2A95EAF797CF8B
:10073000109218011092170188EE93E0A0E0B0E04B
:100740008093190190931A01A0931B01B0931C018F
:1007500084E690E0909316018093150110922C018D
:1007600010922B0110922E0110922D011092300147
:1007700010922F01109232011092310160913301D9
:100780006E7F6D7F609333016695617081E06827AD
:1007900080E0B7DC61E080E0EFDCEFE3F0E0E491E3
:1007A000E0932501E4E3F0E0E491F0E0EE0FFF1FB9
:1007B000E25DFF4F859194919093270180932601EC
:1007C00060E081E0D9DC8091330181FD03C061E00C
:1007D00081E097DC81E080932101E0E4F0E0E491A6
:1007E000E0932201E5E3F0E0E491F0E0EE0FFF1F7B
:1007F000EE5DFF4F859194919093240180932301A6
:10080000089584E690E090931601809315018091FD
:100810001301909114018551914071F4E0912801E8
:10082000F0912901908180912A018095892380830C
:100830001092140110921301089597FB072E16F4DD
:10084000009406D077FD08D00BD007FC05D03EF40D
:10085000909581959F4F0895709561957F4F08956C
:10086000AA1BBB1B51E107C0AA1FBB1FA617B707D6
:1008700010F0A61BB70B881F991F5A95A9F78095F2
:100880009095BC01CD010895EE0FFF1F0590F491E6
:10089000E02D099410E0CCE2D0E003C0FE01F4DFCB
:0C08A0002196CD32D107D1F7F894FFCF9C
:1008AC00000000005F015400F3015300BB01D201B2
:1008BC0047010D0A2B5354574D4F443D300D0A0040
:1008CC000D0A2B53544E413D4D616B6572626C6F3A
:1008DC00636B0D0A000D0A2B53544F4155543D3197
:1008EC000D0A000D0A2B53544155544F3D300D0A3F
:1008FC0000626C7565746F6F746820636F6E6E65E3
:08090C0063746564210A000018
:00000001FF
